:100000008A110A1205280000090007309F00831694
:1000100010308500860183128601850183168511C3
:100020008312851183160511831205110730AE0066
:100030000430AF002D10AD102C10AC102C11AC11F1
:100040002C12AC122C13AC1386018316851183126B
:1000500085150230A000A101EC21831685118312C1
:100060008511051E2C14051A2C100130A000A101C9
:10007000EC2183160511831205150130A000A101A2
:10008000EC218316051183120511051EAC14051A07
:10009000AC100130A000A101EC21831605118312E0
:1000A00005150130A000A101EC2183160511831272
:1000B0000511051E2C17051A2C130130A000A101F3
:1000C000EC2183160511831205150130A000A10152
:1000D000EC218316051183120511051EAC17051AB4
:1000E000AC130130A000A101EC218316051183128D
:1000F00005150130A000A101EC2183160511831222
:100100000511051E2C15051A2C110130A000A101A6
:10011000EC2183160511831205150130A000A10101
:10012000EC218316051183120511051EAC15051A65
:10013000AC110130A000A101EC218316051183123E
:1001400005150130A000A101EC21831605118312D1
:100150000511051E2C16051A2C120130A000A10154
:10016000EC2183160511831205150130A000A101B1
:10017000EC218316051183120511051EAC16051A14
:10018000AC120130A000A101EC212C1FD628AD1C1F
:10019000D328AD102D1CCE282D10D1281F3083055B
:1001A0002D141F3083051F308305D9281F30830588
:1001B000AD141F3083052C1DE6282D1CE1282721B6
:1001C000E4281F308305BA211F3083051F308305C3
:1001D000AC1DF3282D1CEE285821F1281F30830573
:1001E00089211F3083051F3083052C1EF928051334
:1001F00085171F308305AC1EFF28051785131F3098
:1002000083052C1A09291F308305AC1A0929051307
:1002100085131F3083052C1C132985140230A00080
:10022000A101EC2116291F30830585101F3083059D
:10023000AC1C202905140230A000A101EC212329C7
:100240001F30830505101F3083051C282629013027
:1002500086002E08A000A101EC21033086002E08A4
:10026000A000A101EC21023086002E08A000A1010F
:10027000EC21063086002E08A000A101EC210430FC
:1002800086002E08A000A101EC210C3086002E086B
:10029000A000A101EC21083086002E08A000A101D9
:1002A000EC21093086002E08A000A101EC210800F5
:1002B000093086002E08A000A101EC21083086003C
:1002C0002E08A000A101EC210C3086002E08A00011
:1002D000A101EC21043086002E08A000A101EC2130
:1002E000063086002E08A000A101EC210230860015
:1002F0002E08A000A101EC21033086002E08A000EA
:10030000A101EC21013086002E08A000A101EC2102
:100310000800103086002F08A000A101EC21303029
:1003200086002F08A000A101EC21203086002F08B4
:10033000A000A101EC21603086002F08A000A101DF
:10034000EC21403086002F08A000A101EC21C03034
:1003500086002F08A000A101EC21803086002F0824
:10036000A000A101EC21903086002F08A000A1017F
:10037000EC210800903086002F08A000A101EC219C
:10038000803086002F08A000A101EC21C03086003B
:100390002F08A000A101EC21403086002F08A0000A
:1003A000A101EC21603086002F08A000A101EC2102
:1003B000203086002F08A000A101EC2130308600FB
:1003C0002F08A000A101EC21103086002F08A0000A
:1003D000A101EC210800EB29A0080319F729FE214F
:1003E000A00300000000000000000000EC29A108AC
:1003F00003190800FE21A103A003EC290C30A5007D
:10040000A50B002A000000001230A200A20B0D2A4A
:100410000F220F220000000008000F22062A0D30D4
:0A042000A400A40B112A000008003C
:02400E00703F01
:00000001FF
